:100000000C9464000C94AB0E0C94D80E0C948C00E1
:100010000C948C000C948C000C948C000C941F0E8F
:100020000C948C000C948C000C948C000C948C0020
:100030000C948C000C948C000C948C000C948C0010
:100040000C94C2170C948C000C94CC030C94FD03FC
:100050000C948C000C948C000C948C000C948C00F0
:100060000C948C000C948C000200000000240027EB
:10007000002A0000000000250028002B00000000DE
:1000800000230026002900040404040404040402DC
:100090000202020202030303030303010204081025
:1000A00020408001020408102001020408102000F2
:1000B0000000070002010000030406000000000029
:1000C0000000000069053F0611241FBECFEFD8E0F5
:1000D000DEBFCDBF12E0A0E0B1E0E6E1FDE402C08A
:1000E00005900D92A03CB107D9F713E0A0ECB2E067
:1000F00001C01D92AE3AB107E1F710E0C8ECD0E0C4
:1001000004C02297FE010E94B622C43CD107C9F761
:100110000E94EF010C9489260C940000CF93DF938A
:1001200060ED77E080E090E00E944A18C2E6D3E0FC
:10013000CE0160E071E00E94DF0660ED77E080E0D4
:1001400090E00E944A18CE010E946403DF91CF9193
:100150000895CF93DF9386E060E00E946719C2E6BE
:10016000D3E0CE0140E056E960E070E00E948304F5
:10017000CE016BE071E00E94DF06CE0169E171E023
:100180000E94DF06CE0163E371E00E94DF06CE012C
:1001900061E471E00E94DF06CE016FE471E00E942D
:1001A000DF06CE0160E671E00E94DF060E948E004D
:1001B000DF91CF91089584E061E00E94671983E0A8
:1001C00061E00E948B19089584E060E00E94671945
:1001D00083E061E00E948B1908958AE090E00E941C
:1001E000711883E061E00E948B1984E190E00E9425
:1001F000711883E060E00E948B198AE090E00E9411
:10020000711808958AE090E00E94711883E060E020
:100210000E948B1984E190E00E94711883E061E0F4
:100220000E948B198AE090E00E94711808951F9334
:10023000CF93DF9317E0C82FD0E0BE01012E02C09C
:10024000759567950A94E2F7617084E00E948B19B6
:100250000E94ED00115088F784E061E00E948B1944
:100260000E94ED00DF91CF911F91089584E060E03E
:100270000E948B198AE090E00E94711883E061E08F
:100280000E948B198AE090E00E94711884E061E07E
:100290000E948B19089584E061E00E948B1983E02D
:1002A00061E00E948B198AE090E00E94711884E05E
:1002B00060E00E948B198AE090E00E94711883E050
:1002C00060E00E948B198AE090E00E947118089506
:1002D0000F931F938AE090E00E94711817E000E0EE
:1002E00084E00E94C319682F282F30E0012E02C03D
:1002F000220F331F0A94E2F7022B8CE00E948B1925
:100300000E940201115060F70E940201802F1F918C
:100310000F910895EF92FF920F931F938091CB025C
:100320008795882787950091CC02000F000F000F5A
:10033000082B8091CD02082B8091CF028295880FE7
:10034000807E1091D002110F110F110F182B809188
:10035000CE02182B9091D10297959927979580916D
:10036000D5028295807F892B9091D702892B90911D
:10037000D902990F990F990F982BE090D402EE0CA7
:10038000E92A9091D2029795992797958091D30267
:100390008295880F880F807C892B9091D802892BB9
:1003A000F090D602FF0CFF0CF82A0E94DB000E949E
:1003B0004B0188EC0E941701802F0E941701812FAA
:1003C0000E9417018E2D0E9417018F2D0E94170188
:1003D0000E9436011F910F91FF90EF9008958F9228
:1003E0009F92AF92BF92CF92DF92EF92FF920F93C4
:1003F0001F93DF93CF93CDB7DEB727970FB6F8944F
:10040000DEBF0FBECDBF0E947B1885E061E00E9479
:10041000671985E060E00E948B190E94A90082E0C4
:1004200060E00E94671983E061E00E94671986E03E
:1004300060E00E9467198CE061E00E9467198DE01E
:1004400061E00E9467198DE061E00E948B1985E0F0
:1004500061E00E948B196AEF70E080E090E00E94FA
:100460004A180E948A010AEF10E07E010894E11CFC
:10047000F11CA4E0AA2EB12CAC0EBD1EF2E08F2E12
:10048000912C8C0E9D1E82E00E94C3198130910533
:1004900009F0BBC08CE061E00E948B198DE060E048
:1004A0000E948B190E94DB000E944B0189EC0E9484
:1004B000170182E00E94C319009709F0A6C08DE0E1
:1004C00061E00E948B190E94E400E1ECCE2EE2E094
:1004D000DE2E0E946801F60181936F01FBECCF16BE
:1004E000F2E0DF06B1F70E94DB000E943601809146
:1004F000C10289838091C30290E0A0E0B0E0BA2FEE
:10050000A92F982F88272091C40230E040E050E0C6
:10051000822B932BA42BB52B2091C20230E040E01C
:1005200050E02770307040705070A90133272227A7
:10053000822B932BA42BB52B8C839D83AE83BF83FF
:100540008091C602829586958695837090E0209171
:10055000C50230E0220F331F220F331F822B932B53
:100560009B838A8313C082E693E00E944203823019
:1005700029F0833031F0813049F406C00AEF10E0F1
:1005800005C002E310E002C008EE13E082E693E04B
:100590000E9413031816190634F386E00E94C3194B
:1005A0002091C002009759F1222319F481E0809331
:1005B000C00282E693E063E771E042E050E00E940F
:1005C0004E0682E693E062E771E041E050E00E946F
:1005D0004E0682E693E0B70141E050E00E944E06ED
:1005E00082E693E0B50144E050E00E944E0682E6C8
:1005F00093E0B40142E050E00E944E0606C0222380
:1006000021F00E948E001092C002B80180E090E0BC
:100610000E944A188CE060E00E948B198DE060E037
:100620000E948B1930CFFC0184859585FC01E05C2C
:10063000FF4F208131818E5B9F4FFC018081918132
:10064000281B390B2F733070C9010895FC01848574
:100650009585FC01E05CFF4F40815181FC01EE5B20
:10066000FF4F208131814217530741F00190F08103
:10067000E02DE80FF91F208130E002C02FEF3FEF9F
:10068000C9010895FC0184859585FC01E05CFF4F5C
:1006900040815181FC01EE5BFF4F20813181421787
:1006A000530771F0A081B181A80FB91F2C918081EF
:1006B000918101968F7390709183808330E002C0A6
:1006C0002FEF3FEFC9010895DC011E968D919C919B
:1006D0001F97FC01E05CFF4F8E5B9F4F4081518173
:1006E000DC012D913C91119742175307B9F70895FA
:1006F0001F93FC01162F26853785D901A05CBF4FBB
:100700008D919C91019660E470E00E941922D901BC
:10071000AE5BBF4F4D915C91119784179507D1F354
:10072000D901A05CBF4F0D90BC91A02DA20FB31FAB
:100730001C93A685B785A05CBF4F11969C938E93A2
:10074000A689B7892C9181E090E0058C02C0880FC2
:10075000991F0A94E2F7282B2C9381E090E01F91D7
:100760000895FB01E05CFF4F208131812F5F3F4FF7
:100770002F733070DB01AE5BBF4F4D915C911197D1
:100780002417350739F0A081B181A60FB71F8C93CC
:1007900031832083089508951F920F920FB60F9210
:1007A00011242F933F934F935F936F937F938F9376
:1007B0009F93AF93BF93EF93FF938091C6006AED31
:1007C00072E00E94B103FF91EF91BF91AF919F91B1
:1007D0008F917F916F915F914F913F912F910F90EA
:1007E0000FBE0F901F90189582E693E00E941303AE
:1007F000009711F00E94CB0308951F920F920FB63D
:100800000F9211242F933F935F936F937F938F9356
:100810009F93AF93BF93EF93FF9320915E0330912B
:100820005F0380916003909161032817390731F4C9
:100830008091C1008F7D8093C10016C0E09160035C
:10084000F0916103E25EFC4F208180916003909102
:100850006103019660E470E00E94192290936103A5
:10086000809360032093C600FF91EF91BF91AF91F9
:100870009F918F917F916F915F913F912F910F90F9
:100880000FBE0F901F9018958F92AF92BF92CF928C
:10089000DF92EF92FF920F931F93DF93CF93CDB729
:1008A000DEB7FC011382128288EE93E0A0E0B0E094
:1008B00084839583A683B78389E791E091838083BE
:1008C0007587648757874687318B208B138B028B04
:1008D000F58AE48AD78AC68AB18EA08E828E8E85EA
:1008E000838F8F85848F8889858F8989868FCF9123
:1008F000DF911F910F91FF90EF90DF90CF90BF900D
:10090000AF908F9008959F92AF92BF92CF92DF9257
:10091000EF92FF920F931F93CF93DF93EC017A0135
:100920008B0199249394EC89FD8981E090E00E8CF1
:1009300002C0880F991F0A94E2F7808360E874E888
:100940008EE190E0A80197010E942C2221503040B6
:1009500040405040569547953795279590E4A92EED
:1009600092E4B92E9FE0C92ED12C12C09924EC89B3
:10097000FD891082C601B501A80197010E942C22B1
:100980002150304040405040569547953795279527
:1009900080E12030380710F0992041F7E889F98983
:1009A0003083EA89FB892083EE89FF89408181E0D9
:1009B00090E09C010A8C02C0220F331F0A94E2F7D8
:1009C000422B4083EE89FF8940819C010B8C02C041
:1009D000220F331F0A94E2F7422B4083EE89FF89EE
:1009E00040819C010C8C02C0220F331F0A94E2F755
:1009F000422B4083EE89FF8920810D8C02C0880F35
:100A0000991F0A94E2F7809582238083DF91CF912A
:100A10001F910F91FF90EF90DF90CF90BF90AF901C
:100A20009F900895CF93DF93FC0186859785DC0125
:100A3000A05CBF4F8E5B9F4F4D915C911197EC0175
:100A40002881398142175307B9F7A689B7894C9194
:100A500081E090E09C01028C02C0220F331F0A94B7
:100A6000E2F7209524232C93A689B7894C919C0109
:100A7000038C02C0220F331F0A94E2F7209524232F
:100A80002C93A689B7894C919C01048C02C0220F3B
:100A9000331F0A94E2F7209524232C93A689B78963
:100AA0002C91058C02C0880F991F0A94E2F780955B
:100AB00082238C9384859585FC01EE5BFF4F20811A
:100AC0003181805C9F4FFC0131832083DF91CF9186
:100AD0000895109265031092640388EE93E0A0E0FD
:100AE000B0E08093660390936703A0936803B0938C
:100AF0006903E4E6F3E089E791E0929382938AED5B
:100B000092E0958784878EE193E09787868785ECCE
:100B100090E0918B808B84EC90E0938B828B80ECC7
:100B200090E0958B848B81EC90E0978B868B86ECA4
:100B300090E0918F808F84E0828F83E0838F87E0C5
:100B4000848F85E0858F81E0868F08958F929F92B4
:100B5000AF92BF92CF92DF92EF92FF920F931F93CB
:100B6000CF93DF934C017B0182E0A82EB12CA80C1F
:100B7000B91CC0E0D0E0CC24DD24F50161915F0117
:100B8000C7014AE050E00E9403088C01C7016EE2F1
:100B90000E94E206080F191FC00ED11E2196C33015
:100BA000D10559F7C701F40165814AE050E00E9480
:100BB0000308C80ED91EC601DF91CF911F910F9176
:100BC000FF90EF90DF90CF90BF90AF909F908F906D
:100BD0000895FC0189E991E0918380831282138258
:100BE0001482158208950F93FC0189E991E09183A5
:100BF000808362834383248305830F910895FC01DE
:100C000089E991E091838083428353836483758370
:100C10000895FC0189E991E091838083DB012D91A6
:100C20003D914D915C911397228333834483558387
:100C30000895CF93DF93FC01EB0188819981AA810C
:100C4000BB8182839383A483B583CF01DF91CF914E
:100C50000895FC01428353836483758308959B0147
:100C6000BC016E5F7F4FC90144E050E00E944C25FB
:100C70009C0181E02115310509F080E0089589E9A2
:100C800091E09093820380938103109283031092EA
:100C9000840310928503109286030895CF92DF9209
:100CA000EF92FF920F931F93CF93DF936C017B0121
:100CB0008A01C0E0D0E00FC0D7016D917D01D6015F
:100CC000ED91FC910190F081E02DC6010995C80FCE
:100CD000D91F015010400115110571F7CE01DF91A8
:100CE000CF911F910F91FF90EF90DF90CF900895DB
:100CF000DB010D900020E9F7AD0141505040461B4B
:100D0000570BDC01ED91FC910280F381E02D0995F8
:100D10000895EF92FF920F931F93CF93DF937C017F
:100D2000062F172FC0E0D0E0F8010F5F1F4F64912E
:100D3000662351F0F701A081B181ED91FC91C701CB
:100D40000995C80FD91FF0CFCE01DF91CF911F9128
:100D50000F91FF90EF900895AF92BF92CF92DF92E4
:100D6000EF92FF920F931F93CF93DF937C016B0160
:100D7000C0E0D0E000E010E010C0D701ED91FC91A0
:100D8000A080B180C601BE010E947E14682FC701F9
:100D9000F5010995080F191F2196F60184819581A7
:100DA000C817D90750F3C801DF91CF911F910F9158
:100DB000FF90EF90DF90CF90BF90AF9008950E948A
:100DC00078060895DC01ED91FC910190F081E02D11
:100DD000099508959C01CB01DB01ED91FC910190F7
:100DE000F081E02DB901099508950F931F93CF93DA
:100DF000DF93EC016DE00E94E2068C01CE016AE017
:100E00000E94E206080F191FC801DF91CF911F91C0
:100E10000F9108950F931F93CF93DF93EC010E94DE
:100E200089068C01CE010E94F506080F191FC80122
:100E3000DF91CF911F910F9108950F931F93CF933F
:100E4000DF93EC010E94AC068C01CE010E94F506F6
:100E5000080F191FC801DF91CF911F910F910895BD
:100E60000F931F93CF93DF93EC010E9478068C01C0
:100E7000CE010E94F506080F191FC801DF91CF911E
:100E80001F910F9108950F931F93CF93DF93EC0160
:100E90000E94E2068C01CE010E94F506080F191F80
:100EA000C801DF91CF911F910F9108950F931F9368
:100EB000CF93DF93EC010E94EA068C01CE010E94E1
:100EC000F506080F191FC801DF91CF911F910F91EF
:100ED00008958F929F92AF92BF92CF92DF92EF923E
:100EE000FF920F931F93DF93CF93CDB7DEB7A197F8
:100EF0000FB6F894DEBF0FBECDBF6C01042FE52FF7
:100F0000CB01122F19A2223008F41AE021E2E22EBE
:100F1000F12CEC0EFD1E812E9924AA24BB2403C0C3
:100F2000022FE32FCA01602F7E2FA50194010E949A
:100F30002C22129F802D1124081B0894E108F1082F
:100F40000A3014F4005D01C0095CF701008321152B
:100F500031054105510521F7C601B7010E94780608
:100F6000A1960FB6F894DEBF0FBECDBFCF91DF9133
:100F70001F910F91FF90EF90DF90CF90BF90AF90B7
:100F80009F908F9008952115310549F4DC01ED9172
:100F9000FC910190F081E02D642F099508950E9445
:100FA000690708950F931F93CF93DF93EC010E947D
:100FB000C3078C01CE010E94F506080F191FC80156
:100FC000DF91CF911F910F9108959A01AB0160E0DD
:100FD00070E00E94C30708950F931F93CF93DF9390
:100FE000EC019A01AB0160E070E00E94C3078C0144
:100FF000CE010E94F506080F191FC801DF91CF919D
:101000001F910F9108959A01462F50E060E070E023
:101010000E94C30708950F931F93CF93DF93EC01B2
:101020009A01462F50E060E070E00E94C3078C01F7
:10103000CE010E94F506080F191FC801DF91CF915C
:101040001F910F910895CF92DF92EF92FF920F932D
:101050001F93CF93DF93EC017A018B0121153105AA
:1010600041F4E881F9810190F081E02D642F099528
:101070001AC02A303105A9F477FF12C06DE20E9430
:10108000E2066C0144275527BA014E195F09600B2F
:10109000710BCE012AE00E946907C80ED91E04C058
:1010A0002AE00E9469076C01C601DF91CF911F9170
:1010B0000F91FF90EF90DF90CF9008950F931F93C3
:1010C000CF93DF93EC010E9423088C01CE010E9494
:1010D000F506080F191FC801DF91CF911F910F91DD
:1010E00008959A01FB01AF01662757FD6095762FA1
:1010F0000E94230808950F931F93CF93DF93EC0171
:101100009A01CB01AC01662757FD6095762FCE0181
:101110000E9423088C01CE010E94F506080F191FBA
:10112000C801DF91CF911F910F9108956F927F9227
:101130009F92AF92BF92CF92DF92EF92FF920F9366
:101140001F93CF93DF933C017A018B01C22ECB0119
:10115000BA0120E030E0A9010E94B61E87FF0AC054
:10116000C3016DE20E94E206EC0117FB109517F92E
:10117000109502C0C0E0D0E0DD2450E040E030E057
:101180002FE311C0DA01F9016B2F742F8F2F922FEB
:1011900020E030E040E251E40E94D81D562F472F56
:1011A000382F292FD394DC1468F3C801B701DA0172
:1011B000F9012B2F342F4F2F5E2F0E94801C5B01D3
:1011C000F82E992E7B2D0E940A1B162FD72EE82E63
:1011D000092F0E94981F9B01AC016A2D7B2D8F2D3A
:1011E000992D0E94AD1C962EA72EB82EF92EC30164
:1011F000412F5D2D6E2D702F2AE030E00E94C30735
:10120000C80FD91FCC20B9F1C30161EA71E00E9477
:101210007806C80FD91F2FC0692D7A2D8B2D9F2DD1
:1012200020E030E040E251E40E94DE1CD62EB72ED2
:10123000A82E992E0E94461F7B010027F7FC0095DF
:10124000102FC301B801A7012AE030E00E94230853
:10125000C80FD91FC801B7010E94E61E9B01AC014F
:101260006D2D7B2D8A2D992D0E94AD1C962EA72EBB
:10127000B82EF92ECA94CC2079F6CE01DF91CF9109
:101280001F910F91FF90EF90DF90CF90BF90AF90A4
:101290009F907F906F9008950E94960808950F93F5
:1012A0001F93CF93DF93EC010E9496088C01CE012F
:1012B0000E94F506080F191FC801DF91CF911F91F9
:1012C0000F910895CF93DF93EC010E941618688761
:1012D00079878A879B87E881F9810680F781E02DED
:1012E000CE0109959C0197FF15C00E94161828850C
:1012F00039854A855B85621B730B840B950B2C81AA
:101300003D814E815F81621773078407950718F34B
:101310002FEF3FEFC901DF91CF910895CF93DF9376
:10132000EC010E941618688779878A879B87E88175
:10133000F9810084F185E02DCE0109959C0197FF8C
:1013400015C00E941618288539854A855B85621B61
:10135000730B840B950B2C813D814E815F8162174D
:1013600073078407950718F32FEF3FEFC901DF914B
:10137000CF910895CF93DF93EC01CE010E948E09A7
:101380009C0197FD0FC08D32910561F0C0978A30A6
:10139000910540F0E881F9810680F781E02DCE01CA
:1013A0000995EBCFC901DF91CF910895FC014483EA
:1013B00055836683778308956F927F928F929F9271
:1013C000AF92BF92CF92DF92EF92FF920F931F9353
:1013D000CF93DF933C016B014A0159017801FB0176
:1013E0008081882391F1C0E0D0E000E010E026C0C9
:1013F000F601E00FF11F2081332727FD309582177A
:10140000930731F40F5F1F4F0815190518F01DC021
:1014100000E010E0E114F10479F0F501EC0FFD1F9C
:101420002081332727FD30958217930729F42196D1
:10143000CE15DF0518F00BC0C0E0D0E0C3010E945C
:10144000620918161906A4F202C081E001C080E00A
:10145000DF91CF911F910F91FF90EF90DF90CF9090
:10146000BF90AF909F908F907F906F9008950F9353
:101470001F93CF93DF939A01FB0101900020E9F7BE
:101480003197E61BF70BEA0109900020E9F78E017E
:1014900001501040041B150BAF010E94DC09DF91C5
:1014A000CF911F910F91089540E050E00E94370ABC
:1014B00008950F931F9320E030E000E010E00E94B9
:1014C000DC091F910F9108959F92AF92BF92CF9226
:1014D000DF92EF92FF920F931F93CF93DF936C01F4
:1014E000A62E0E94BA09EC0197FD4EC0EE24FF24FF
:1014F00087019924BB24A7FCB094CA15DB0531F100
:10150000CD32D10509F1CE01C0978A309105F0F4B2
:10151000C801B7012AE030E040E050E00E94FA2123
:101520007B018C01CE01AA2797FDA095BA2FE80E6A
:10153000F91E0A1F1B1F80ED9FEFAFEFBFEFE80EF4
:10154000F91E0A1F1B1F02C099249394D601ED9126
:10155000FC910680F781E02DC6010995C6010E9425
:101560008E09EC01C0978A30910538F2CA15DB0567
:1015700021F2992061F010950095F094E094E11C1F
:10158000F11C011D111D03C0EE24FF248701B701CA
:10159000C801DF91CF911F910F91FF90EF90DF90E5
:1015A000CF90BF90AF909F90089561E00E94640A31
:1015B00008956F927F928F929F92AF92BF92CF9237
:1015C000DF92EF92FF920F931F93CF93DF93EC0183
:1015D000762E0E94BA09D82E87FD7DC0BB24AA248E
:1015E00090E8992E8FE3882EEE24FF248701CC24E7
:1015F0006624D714E1F18D2D8D32A1F18E32A9F13F
:1016000080538A30A0F5C801B7012AE030E040E0FD
:1016100050E00E94FA217B018C018D2D992787FDD6
:101620009095A92FB92FE80EF91E0A1F1B1F80EDF8
:101630009FEFAFEFBFEFE80EF91E0A1F1B1FCC2074
:10164000B1F0A5019401652F7A2D832F982D2DECF3
:101650003CEC4CEC5DE30E94DE1CB62EA72E982ECF
:10166000892E05C06624639402C0CC24C394E8810B
:10167000F9810680F781E02DCE010995CE010E9407
:101680008E09D82E982F90539A3008F4B2CF8E320C
:1016900009F4AFCF871509F4ACCF662041F010955F
:1016A0000095F094E094E11CF11C011D111DCC206B
:1016B00069F0C801B7010E94E61ED501F4012B2F85
:1016C0003A2D4F2F582D0E94DE1C09C0C801B701CA
:1016D0000E94E61E04C060E070E080E090E0DF91D0
:1016E000CF911F910F91FF90EF90DF90CF90BF901F
:1016F000AF909F908F907F906F90089561E00E94CF
:10170000D90A0895CF92DF92EF92FF920F931F9321
:10171000CF93DF936C01EB017A0100E010E008C089
:10172000C6010E94620997FD06C089930F5F1F4F93
:101730000E151F05A8F3C801DF91CF911F910F91DE
:10174000FF90EF90DF90CF900895AF92BF92CF922D
:10175000DF92EF92FF920F931F93CF93DF935C0181
:10176000EA01790121153105B1F000E010E0C62E43
:10177000DD24C7FCD0940BC0C5010E94620997FD0F
:101780000CC08C159D0549F089930F5F1F4F0E15F6
:101790001F0590F302C000E010E0C801DF91CF9177
:1017A0001F910F91FF90EF90DF90CF90BF90AF907F
:1017B00008952F923F924F925F926F927F928F92F5
:1017C0009F92AF92BF92DF92EF92FF920F931F937F
:1017D000DF93CF9300D000D0CDB7DEB71B012983B4
:1017E0003A834B835C839091AB01981721F09F3F24
:1017F00009F0D8C104C0E8E6F0E0D4907DC0809341
:10180000AB01E8E6F0E0D4909D2D9F3F09F4CAC1FA
:10181000913031F1923009F449C0DD2009F06CC0FB
:1018200014BC15BC94B5926094BD95B5916095BDFE
:10183000282F30E0F901E957FF4FE491F0E0EE0F77
:10184000FF1FED58FF4F4591549140938B035093E8
:101850008C0325563F4FF901249120938D034EC0F0
:101860001092800010928100909181009860909376
:10187000810090918100916090938100282F30E049
:10188000F901E957FF4FE491F0E0EE0FFF1FED582B
:10189000FF4F4591549140939203509393032556E3
:1018A0003F4FF90124912093940328C01092B00077
:1018B0001092B1009091B00092609093B00090911E
:1018C000B10091609093B100282F30E0F901E95701
:1018D000FF4FE491F0E0EE0FFF1FED58FF4F4591F1
:1018E00054914093990350939A0325563F4FF90121
:1018F000249120939B0302C0D7FC54C161E00E9455
:101900006719DD2021F0FD2DF23009F0C1C0410141
:10191000AA24BB2460E079E08DE390E0A501940166
:101920000E942C2229013A0179018A010894E108D8
:10193000F108010911098FEFE816F10401051105FD
:1019400009F008F498C060E271EA87E090E0A50130
:1019500094010E942C2279018A010894E108F1087F
:10196000010911099D2D9230C9F4AFEFEA16F10477
:101970000105110509F008F485C068E478EE81E0FE
:1019800090E0A50194010E942C2279018A0108941B
:10199000E108F1080109110983E001C082E0BFEF0D
:1019A000EB16F1040105110509F008F465C064E2C5
:1019B00074EF80E090E0A50194010E942C2279014F
:1019C0008A010894E108F10801091109DD20E1F01C
:1019D000ED2DE230D9F4FFEFEF16F104010511050A
:1019E00009F008F451C062E17AE780E090E0A501D7
:1019F00094010E942C2279018A010894E108F108DF
:101A00000109110985E003C083E001C084E09FEF74
:101A1000E916F1040105110579F170F169E07DE342
:101A200080E090E0A50194010E942C2279018A01B6
:101A30000894E108F10801091109DD2011F484E09E
:101A400001C086E0AFEFEA16F10401051105A1F02F
:101A500098F0830172019AE016950795F794E79440
:101A60009A95D1F70894E108F10801091109DD20E0
:101A700031F087E00AC081E0DD2011F006C085E08A
:101A800085BD3CC082E001C084E08093B10036C0D7
:101A90004101AA24BB2460E079E08DE390E0A50138
:101AA00094010E942C2279018A010894E108F1082E
:101AB00001091109B0E0EB16B0E0FB06B1E00B073D
:101AC000B0E01B0788F064E274EF80E090E0A501CD
:101AD00094010E942C2279018A010894E108F108FE
:101AE0000109110993E001C091E0ED2DE13031F4DD
:101AF00080918100887F892B8093810089819A81E0
:101B0000AB81BC810097A105B10591F0B101660FD1
:101B1000771F80E090E029813A814B815C810E94AF
:101B2000FA2128EE33E040E050E00E942C2203C06E
:101B30002FEF3FEFA9019D2D913099F0923019F1CF
:101B4000DD2081F5E7BC2093870330938803409321
:101B5000890350938A0380916E00826080936E00A7
:101B600021C0F0928900E092880020938E03309388
:101B70008F03409390035093910380916F00826094
:101B800080936F000FC0E092B300209395033093D1
:101B9000960340939703509398038091700082605E
:101BA000809370000F900F900F900F90CF91DF9166
:101BB0001F910F91FF90EF90DF90BF90AF909F909B
:101BC0008F907F906F905F904F903F902F900895EF
:101BD000813041F0813018F08230D1F409C0109288
:101BE0006E00089580916F008D7F80936F0008953F
:101BF000809170008D7F8093700081E08093B000B1
:101C00008091B100887F84608093B1001092B3000E
:101C100008951F93182F8091AB01811739F4E8E6DE
:101C2000F0E084919FEF9093AB0101C08FEF0E9491
:101C3000E80D812F60E00E948B191F9108951F927B
:101C40000F920FB60F9211242F933F934F935F93F0
:101C50006F937F938F939F93AF93BF93EF93FF9374
:101C60008091950390919603A0919703B09198036A
:101C70000097A105B10551F1E0919903F0919A0304
:101C8000808190919B038927808380919503909117
:101C90009603A0919703B0919803181619061A0697
:101CA0001B06C4F48091950390919603A09197032D
:101CB000B09198030197A109B1098093950390937E
:101CC0009603A0939703B093980304C08091AB014F
:101CD0000E94090EFF91EF91BF91AF919F918F915B
:101CE0007F916F915F914F913F912F910F900FBE18
:101CF0000F901F9018958230E8F4E82FF0E0EE0F77
:101D0000FF1FE456FC4F71836083813041F0809166
:101D100069008C7F842B80936900E89A08958091F4
:101D20006900440F551F440F551F837F842B8093F8
:101D30006900E99A0895823068F4813011F0E898DA
:101D400001C0E998E82FF0E0EE0FFF1FE456FC4FCA
:101D50001182108208951F920F920FB60F921124D4
:101D60002F933F934F935F936F937F938F939F93A3
:101D7000AF93BF93EF93FF9380919C0390919D034A
:101D8000009729F0E0919C03F0919D030995FF9144
:101D9000EF91BF91AF919F918F917F916F915F91E3
:101DA0004F913F912F910F900FBE0F901F9018955C
:101DB0001F920F920FB60F9211242F933F934F93C0
:101DC0005F936F937F938F939F93AF93BF93EF93A3
:101DD000FF9380919E0390919F03009729F0E091DB
:101DE0009E03F0919F030995FF91EF91BF91AF91F1
:101DF0009F918F917F916F915F914F913F912F9123
:101E00000F900FBE0F901F901895009729F0BC01FE
:101E100080E090E00E9439240895EF92FF920F93A2
:101E20001F937B018C01611571058105910549F0B6
:101E30000E943424A80197010E944E229B01AC010C
:101E400003C020E030E0A901B901CA011F910F9140
:101E5000FF90EF900895EF92FF920F931F937B01F5
:101E60008C01621773078407950764F4CA01B901EE
:101E70006E197F09800B910B0E940D0FE60EF71E65
:101E8000081F191FB701C8011F910F91FF90EF9014
:101E900008952F923F924F925F926F927F928F920E
:101EA0009F92AF92BF92CF92DF92EF92FF920F93E9
:101EB0001F93DF93CF93CDB7DEB73B014C011901E0
:101EC0002A016D897E898F89988D6A197B098C0911
:101ED0009D09621A730A840A950AA40193010E945B
:101EE000FA21E218F30804091509A80197010E94D4
:101EF0004E222A0D3B1D4C1D5D1DB901CA01CF911B
:101F0000DF911F910F91FF90EF90DF90CF90BF90E6
:101F1000AF909F908F907F906F905F904F903F9089
:101F20002F900895089570E0382F20E0622B732BD6
:101F3000CB010895FC01808191810E945423089572
:101F4000CF93DF93EC0188819981009711F00E9473
:101F50005423198218821D821C821B821A82DF91EF
:101F6000CF9108950F931F93CF93DF93EC018B01D3
:101F70006F5F7F4F888199810E944224009731F0E2
:101F8000998388831B830A8381E001C080E0DF910D
:101F9000CF911F910F910895CF93DF93EC0188812A
:101FA0009981009729F08A819B818617970778F499
:101FB000CE010E94B20F882341F08C819D81009751
:101FC00031F4E881F981108202C080E001C081E033
:101FD000DF91CF910895EF92FF920F931F93CF93CC
:101FE000DF93EC017B018A01BA010E94CC0F8823A8
:101FF00021F4CE010E94A00F07C01D830C838881AD
:102000009981B7010E948825CE01DF91CF911F9160
:102010000F91FF90EF900895CF93DF93FC01118211
:102020001082138212821582148216826115710544
:1020300059F0EB0109900020E9F7AE014150504002
:10204000461B570B0E94EB0FDF91CF910895EF9243
:10205000FF92CF93DF93EC01FB018617970761F0A6
:10206000608171816115710529F0448155810E945B
:10207000EB0F02C00E94A00FCE01DF91CF91FF9025
:10208000EF900895FC011182108213821282158252
:10209000148216820E94271008950F931F938C01BB
:1020A0006115710561F0DB010D900020E9F7AD01CC
:1020B00041505040461B570B0E94EB0F02C00E943C
:1020C000A00FC8011F910F910895EF92FF920F93F7
:1020D0001F93DF93CF93CDB7DEB7A1970FB6F894D8
:1020E000DEBF0FBECDBF7C01CB01BA01F70111826B
:1020F0001082138212821582148216828E010F5F63
:102100001F4FA80130E00E943B26C701B8010E9482
:102110004D10A1960FB6F894DEBF0FBECDBFCF9184
:10212000DF911F910F91FF90EF900895EF92FF9232
:102130000F931F93DF93CF93CDB7DEB7A2970FB660
:10214000F894DEBF0FBECDBF7C01CB01BA01F70111
:1021500011821082138212821582148216828E01DD
:102160000F5F1F4FA80130E00E94F225C701B801A0
:102170000E944D10A2960FB6F894DEBF0FBECDBFE1
:10218000CF91DF911F910F91FF90EF900895EF9203
:10219000FF920F931F93DF93CF93CDB7DEB7619775
:1021A0000FB6F894DEBF0FBECDBF7C01CB01F701A7
:1021B00011821082138212821582148216828E017D
:1021C0000F5F1F4FB80150E00E946026C701B801A1
:1021D0000E944D1061960FB6F894DEBF0FBECDBFC2
:1021E000CF91DF911F910F91FF90EF900895EF92A3
:1021F000FF920F931F93DF93CF93CDB7DEB7629714
:102200000FB6F894DEBF0FBECDBF7C01CB01F70146
:1022100011821082138212821582148216828E011C
:102220000F5F1F4FB80150E00E94D125C701B801D0
:102230000E944D1062960FB6F894DEBF0FBECDBF60
:10224000CF91DF911F910F91FF90EF900895EF9242
:10225000FF920F931F93DF93CF93CDB7DEB72997EC
:102260000FB6F894DEBF0FBECDBF7C01862FF701FD
:10227000118210821382128215821482168290E0DB
:102280008E010F5F1F4FB80150E00E946026C7010A
:10229000B8010E944D1029960FB6F894DEBF0FBE0C
:1022A000CDBFCF91DF911F910F91FF90EF900895D7
:1022B000DF93CF9300D0CDB7DEB7FC01118210823F
:1022C0001382128215821482168269831A82BE01D9
:1022D0006F5F7F4F0E944D100F900F90CF91DF9155
:1022E0000895EF92FF920F931F93CF93DF93EC012A
:1022F0007B010C811D8161157105B9F041155105F6
:1023000091F0040F151FB8010E94CC0F882369F0CB
:10231000288139818C819D81820F931FB7010E9492
:1023200088251D830C8381E001C080E0DF91CF917F
:102330001F910F91FF90EF900895FB0160817181D3
:10234000448155810E94711108956115710561F0F4
:10235000DB010D900020E9F7AD0141505040461BD4
:10236000570B0E947111089580E00895DF93CF9379
:1023700000D0CDB7DEB769831A82BE016F5F7F4F91
:1023800041E050E00E9471110F900F90CF91DF91CA
:102390000895EF92FF920F931F93DF93CF9300D096
:1023A00000D0CDB7DEB77C01862F90E08E010F5FA5
:1023B0001F4FB8014AE050E00E94D125F80101907A
:1023C0000020E9F7AF0141505040401B510BC701BD
:1023D000B8010E9471110F900F900F900F90CF9144
:1023E000DF911F910F91FF90EF900895EF92FF9270
:1023F0000F931F93DF93CF93CDB7DEB727970FB619
:10240000F894DEBF0FBECDBF7C01CB018E010F5F04
:102410001F4FB8014AE050E00E94D125F801019019
:102420000020E9F7AF0141505040401B510BC7015C
:10243000B8010E94711127960FB6F894DEBF0FBE47
:10244000CDBFCF91DF911F910F91FF90EF90089535
:10245000EF92FF920F931F93DF93CF9300D000D0A2
:1024600000D0CDB7DEB77C01CB018E010F5F1F4FCF
:10247000B8014AE050E00E946026F8010190002077
:10248000E9F7AF0141505040401B510BC701B80163
:102490000E94711126960FB6F894DEBF0FBECDBF15
:1024A000CF91DF911F910F91FF90EF900895EF92E0
:1024B000FF920F931F93DF93CF93CDB7DEB72C9787
:1024C0000FB6F894DEBF0FBECDBF7C01CB01BA01C1
:1024D0008E010F5F1F4FA8012AE030E00E94F22515
:1024E000F80101900020E9F7AF0141505040401B36
:1024F000510BC701B8010E9471112C960FB6F894C8
:10250000DEBF0FBECDBFCF91DF911F910F91FF9026
:10251000EF900895EF92FF920F931F93DF93CF9365
:10252000CDB7DEB72B970FB6F894DEBF0FBECDBF89
:102530007C01CB01BA018E010F5F1F4FA8012AE079
:1025400030E00E943B26F80101900020E9F7AF013E
:1025500041505040401B510BC701B8010E947111FE
:102560002B960FB6F894DEBF0FBECDBFCF91DF9193
:102570001F910F91FF90EF9008950F931F938C017F
:10258000FB0160817181448155810E947111882312
:1025900019F4C8010E94A00FC8011F910F9108955E
:1025A0000F931F938C016115710569F0DB010D908C
:1025B0000020E9F7AD0141505040461B570B0E94E7
:1025C0007111882319F4C8010E94A00FC8011F913E
:1025D0000F9108950F931F938C010E94B6118823C9
:1025E00019F4C8010E94A00FC8011F910F9108950E
:1025F0000F931F938C010E94C911882319F4C801FD
:102600000E94A00FC8011F910F9108950F931F936F
:102610008C010E94F611882319F4C8010E94A00FB2
:10262000C8011F910F9108950F931F938C010E9471
:102630002812882319F4C8010E94A00FC8011F9115
:102640000F9108950F931F938C010E9457128823B6
:1026500019F4C8010E94A00FC8011F910F9108959D
:102660000F931F938C010E948A12882319F4C801CA
:102670000E94A00FC8011F910F910895CF93DF937F
:10268000FC01DB0180819181009731F06D917C919B
:10269000119761157105E9F4CD91DC91119720979F
:1026A00069F014962D913C9115972115310531F063
:1026B000288130E0309521953F4F12C0009771F08E
:1026C000248135812115310549F0FC01208130E05C
:1026D00007C00E947F25282F392F02C020E030E05C
:1026E000C901DF91CF910895FC0144815581FB011F
:1026F000248135814217530729F40E943E1321E0BB
:10270000009709F020E0822F0895FC0184819581D3
:10271000009741F46115710519F081E0FB0109C0D2
:1027200081E008950190F081E02D6115710531F48B
:1027300081E09081992359F080E00895CF010E94B3
:102740007F259C0181E02115310509F080E0089585
:102750000E943E13892F881F8827881F08950E9492
:102760003E1321E0181619060CF020E0822F089580
:102770000E943E1321E0181619060CF420E0822F67
:1027800008950E943E13892F8095881F8827881FEF
:102790000895EF92FF920F931F93CF93DF93FC0165
:1027A000DB018617970729F18481958114962D9175
:1027B0003C91159782179307F1F40097D1F00081AF
:1027C0001181CD91DC9111970FC0992787FD9095CC
:1027D0000E943C257C018991992787FD90950E9454
:1027E0003C25E816F90639F4F80181918F01882318
:1027F00061F781E001C080E0DF91CF911F910F91DF
:10280000FF90EF900895FC01DB01CA0114964D91F1
:102810005C91159724813581241B350B28173907C6
:10282000A0F0208131812115310579F06D917C91E5
:1028300011976115710559F0820F931F0E948F2522
:102840009C0181E02115310519F080E0089580E0B8
:102850000895FC0144815581FB0124813581421793
:10286000530728F040E050E00E940314089580E0F0
:102870000895FC01DB018481958114964D915C9152
:10288000159784179507B0F0208131812115310506
:1028900089F06D917C9111976115710569F0841B28
:1028A000950B820F931F0E947F259C0181E02115CB
:1028B000310519F080E0089580E00895FC018481DD
:1028C00095816817790730F40190F081E02DE60FCB
:1028D000F71F40830895FC0184819581681779076B
:1028E00020F480819181009729F41092A00360EA7E
:1028F00073E002C0680F791FCB010895FC01848149
:1029000095816817790748F480819181009739F0A3
:10291000680F791FFB018081089580E0089580E0B1
:1029200008950E947E1408950F931F93CF93DF9311
:10293000FC018B0141155105F1F061157105D9F0CC
:10294000C481D5812C173D0718F0FB01108213C0FC
:1029500041505040C21BD30B4C175D0708F4EA01ED
:1029600060817181620F731FC801AE010E949D25B5
:10297000C00FD11F1882DF91CF911F910F91089541
:10298000CF93DF93FC01CA0124813581421753079D
:1029900078F4C081D181772767FD70958C0F9D1FDA
:1029A0000E947425009721F09C012C1B3D0B02C056
:1029B0002FEF3FEFC901DF91CF91089540E050E044
:1029C0000E94C0140895CF93DF93FC01CA012481B3
:1029D00035814217530778F4C081D181FB016081B2
:1029E00071818C0F9D1F0E94B725009721F09C01DB
:1029F0002C1B3D0B02C02FEF3FEFC901DF91CF91A0
:102A0000089540E050E00E94E3140895DF92EF92B1
:102A1000FF920F931F93CF93DF93EC018C819D81E5
:102A200048175907F8F47A010894E11CF11CE88171
:102A3000F981EE0DFF1DD080108208811981772762
:102A400067FD7095C8010E94AC250E0D1F1DF80191
:102A5000D082009739F028813981AC01421B530B99
:102A60009A0102C02FEF3FEFC901DF91CF911F9173
:102A70000F91FF90EF90DF900895FC014481558104
:102A8000415050400E9406150895AF92BF92CF92D8
:102A9000DF92EF92FF920F931F93CF93DF93FC018E
:102AA0006B018A01DB0114962D913C91159721153C
:102AB000310551F184819581009731F18217930797
:102AC00018F14817590718F08C0101501040E080A8
:102AD000F180C701CFEFDFEF5701A00EB11E10C08C
:102AE000F601608171810E94B725009779F09C0101
:102AF0002E193F090217130708F49E010196E901F8
:102B0000A816B90668F702C0CFEFDFEFCE01DF915C
:102B1000CF911F910F91FF90EF90DF90CF90BF90DA
:102B2000AF900895FC0144815581FB0124813581DA
:102B3000421B530B0E9445150895AF92BF92CF924E
:102B4000DF92EF92FF920F931F93CF93DF93F82EB4
:102B5000E92E6B018A01E9012417350748F4342F67
:102B6000212F8E01C901A92EE5015E01B22EE501DA
:102B70008F2D9E2D6CEA71E00E940C10D6011496E8
:102B80008D919C91159780179107D8F08C179D0710
:102B900008F4EC01D601ED91FC911197EC0FFD1FAB
:102BA000B08010826D917C91600F711F8F2D9E2DD2
:102BB0000E944D10D601ED91FC911197EC0FFD1F75
:102BC000B0828F2D9E2DDF91CF911F910F91FF909D
:102BD000EF90DF90CF90BF90AF900895CF93DF93A9
:102BE000EC01FB01248135810E949D15CE01DF910E
:102BF000CF910895DC01ED91FC911197309729F464
:102C00000895861709F44083319680818823C9F797
:102C100008952F923F924F925F926F927F928F9280
:102C20009F92AF92BF92CF92DF92EF92FF920F935B
:102C30001F93CF93DF937C012B016A01DC01149673
:102C40006D907C9015976114710409F4D9C0FB0153
:102C5000848095808114910409F4D2C0DA0114961D
:102C6000AD90BC901597A818B908FC01008111819E
:102C7000A114B104F1F413C0D6016C9111967C91AA
:102C8000119714964D915C911597CE010E9459258C
:102C9000D60114960D911C9115970C0F1D1FF20172
:102CA00060817181C8010E94B725EC01009721F76E
:102CB000A7C0B7FC02C0E30142C048012DC0E30138
:102CC000C01BD10BC401B801AE010E945925C80D2B
:102CD000D91DD6016C9111967C91119714964D9146
:102CE0005C911597CE010E945925D60114968D90BE
:102CF0009C9015978C0E9D1EF20104811581060D86
:102D0000171DD70114968D919C9115978A0D9B1DC7
:102D100015969C938E931497F20160817181C8017E
:102D20000E94B7253C01009751F6C401B8010E94EA
:102D3000882566C08C01080D191DCA0DDB1DD20146
:102D40006D917C91C8010E94B725009799F7C6152F
:102D5000D70509F455C0F701828193818C179D072F
:102D600008F045C0C701BE010E94B20F882309F4D4
:102D700047C03DC0C701B201A9010E944515EC0141
:102D800097FD3EC0D7016D917C911197F20184812E
:102D900095818C0F9D1F680F791F14964D915C9142
:102DA0001597481B590BCB018A0D9B1D0E9462256C
:102DB000D70114968D919C9115978A0D9B1D1596A0
:102DC0009C938E931497ED91FC911197E80FF91F46
:102DD00010822D913C912C0F3D1FF6016081718175
:102DE00044815581C9010E9459259E0105C0D70122
:102DF00014962D913C9115972150304037FFBACF52
:102E0000DF91CF911F910F91FF90EF90DF90CF90C6
:102E1000BF90AF909F908F907F906F905F904F90FA
:102E20003F902F900895CF93DF93FC01C081D18113
:102E3000209739F409C0992787FD90950E943C2579
:102E4000899388818823B9F7DF91CF910895CF9333
:102E5000DF93FC01C081D181209739F409C0992703
:102E600087FD90950E944425899388818823B9F72E
:102E7000DF91CF910895AF92BF92CF92DF92EF9200
:102E8000FF920F931F93CF93DF936C01DC01ED90C2
:102E9000FC901197E114F10409F443C01496AD902D
:102EA000BC901597A114B104E1F18701E801888174
:102EB0000F5F1F4F992787FD90950E94342500973B
:102EC000A9F78501015010400E0D1F1DF8018081EA
:102ED000992787FD90950E943425009731F00C17B3
:102EE0001D0718F001501040F1CF0F5F1F4F0C1B52
:102EF0001D0BD60115961C930E931497EC16FD0628
:102F000028F4C701BE01A8010E945925D601ED9100
:102F1000FC91119714968D919C911597E80FF91FCC
:102F20001082DF91CF911F910F91FF90EF90DF9072
:102F3000CF90BF90AF900895FC0180819181009760
:102F400029F00E940D259B01AC0103C020E030E078
:102F5000A901B901CA0108950E94BA2208950E94E8
:102F60005423089521E030E0FC018081882311F092
:102F700020E030E0C901089521E0FC01208308959C
:102F8000089508951F920F920FB60F9211242F9358
:102F90003F934F935F936F937F938F939F93AF93E1
:102FA000BF932091A5033091A6034091A7035091B0
:102FB000A8037091A903DA01C9010296A11DB11DF0
:102FC000672F6A5F6D3730F06D57DA01C9010396DC
:102FD000A11DB11D6093A9038093A5039093A6033F
:102FE000A093A703B093A8038091A1039091A2039B
:102FF000A091A303B091A4030196A11DB11D8093DC
:10300000A1039093A203A093A303B093A403BF9141
:10301000AF919F918F917F916F915F914F913F9170
:103020002F910F900FBE0F901F9018958FB7F894A7
:103030002091A5033091A6034091A7035091A803C6
:103040008FBFB901CA0108959FB7F8942091A103D9
:103050003091A2034091A3035091A40386B5A89B8D
:1030600006C08F3F21F02F5F3F4F4F4F5F4F9FBFF5
:10307000542F432F322F2227280F311D411D511D60
:1030800083E0220F331F441F551F8A95D1F7B901E2
:10309000CA010895EF92FF920F931F93CF93DF938E
:1030A0007B018C010E942418EB010FC00E942418A0
:1030B0006C1B7D0B83E0683E780738F00894E108CC
:1030C000F10801091109C851DC4FE114F1040105AF
:1030D000110561F7DF91CF911F910F91FF90EF9054
:1030E0000895019739F0019729F0880F991F0197EA
:1030F0000197F1F70895789484B5826084BD84B512
:10310000816084BD85B5826085BD85B5816085BDE2
:10311000EEE6F0E0808181608083E1E8F0E01082FB
:10312000808182608083808181608083E0E8F0E03C
:10313000808181608083E1EBF0E080818460808326
:10314000E0EBF0E0808181608083EAE7F0E080815D
:1031500084608083808182608083808181608083BD
:103160008081806880831092C10008958093AD01B2
:1031700008958E3008F08E5087709091AD01929531
:10318000990F990F907C982B90937C0080917A00F6
:10319000806480937A0080917A0086FDFCCF209134
:1031A000780030917900932F80E030E0282B392B84
:1031B000C90108951F93CF93DF93182FEB0161E0AE
:1031C0000E946719209709F44AC0CF3FD10509F43E
:1031D00049C0E12FF0E0E155FF4FE491E330C1F049
:1031E000E43028F4E13051F0E230B1F50CC0E630C3
:1031F00019F1E73049F1E43079F514C084B58068FD
:1032000084BDC7BD33C084B5806284BDC8BD2EC037
:1032100080918000806880938000D0938900C09363
:10322000880024C080918000806280938000D093C9
:103230008B00C0938A001AC08091B0008068809390
:10324000B000C093B30012C08091B0008062809340
:10325000B000C093B4000AC0C038D1051CF4812F5F
:1032600060E002C0812F61E00E948B19DF91CF9155
:103270001F910895833071F0843028F48130A1F0DB
:10328000823021F514C08630B1F08730D1F084301F
:10329000E9F404C0809180008F7703C080918000A2
:1032A0008F7D80938000089584B58F7702C084B5A8
:1032B0008F7D84BD08958091B0008F778093B0009A
:1032C00008958091B0008F7D8093B000089590E0C4
:1032D000FC01E556FF4F2491FC01E957FF4FE491B3
:1032E000EE23C1F0F0E0EE0FFF1FE759FF4F85918D
:1032F0009491DC01662341F49FB7F8948C9120955A
:1033000082238C939FBF08959FB7F8948C91822B52
:103310008C939FBF08950F931F93DF93CF930F92CA
:10332000CDB7DEB7282F30E0F901E155FF4F84918A
:10333000F901E556FF4F149129573F4FF9010491C8
:103340000023D9F0882321F069830E943A1969810A
:10335000E02FF0E0EE0FFF1FED58FF4F85919491A5
:10336000DC019FB7F894662321F48C91109581239A
:1033700002C08C91812B8C939FBF0F90CF91DF91D6
:103380001F910F9108950F931F93282F30E0F9019B
:10339000E155FF4F8491F901E556FF4F04912957FC
:1033A0003F4FF9011491112391F0882311F00E94ED
:1033B0003A19E12FF0E0EE0FFF1FE358FF4F859120
:1033C0009491DC018C91802321E030E011F420E025
:1033D00030E0C9011F910F9108958F929F92AF9293
:1033E000BF92CF92DF92EF92FF920F931F9390E0E4
:1033F000FC01E556FF4F949089579F4FFC01E490E4
:10340000662311F4882401C0892CCA01B90120E483
:103410003FE140E050E00E94FA2120E83EE340E036
:1034200050E00E942C2259016A0180E090E0DC010A
:103430006E2D70E0FB01EE0FFF1FE358FF4F25914B
:10344000349109C08A159B05AC05BD0509F44DC032
:103450000196A11DB11DF90140814921481591F343
:103460000AC08A159B05AC05BD0509F43EC001964E
:10347000A11DB11D07C0660F771F63587F4FFB0169
:1034800025913491F90140814921481551F720E0F7
:1034900030E0A901FB01659174910FC079018A01A7
:1034A000E80EF91E0A1F1B1FEA14FB040C051D057C
:1034B000E1F02F5F3F4F4F4F5F4FFB01E081E9216C
:1034C000E81561F3CA01B90128E032E540E050E0B7
:1034D0000E94FA216058714C8F4F9F4F20E43FE1CA
:1034E00040E050E00E942C2203C020E030E0A9011F
:1034F000B901CA011F910F91FF90EF90DF90CF901B
:10350000BF90AF909F908F900895CF92DF92EF92EF
:10351000FF920F931F93CF93DF93E82EF62EC42EC6
:10352000C7E0D0E0DD2407E010E08F2D61E00E94CD
:103530008B19CC2071F48E2D0E94C31998012C1B7D
:103540003D0BAC0102C0440F551F2A95E2F79A01CA
:103550000AC08E2D0E94C3199C010C2E02C0220F9E
:10356000331F0A94E2F7D22A8F2D60E00E948B1954
:1035700021975FEFCF3FD507C1F68D2DDF91CF911A
:103580001F910F91FF90EF90DF90CF900895BF9221
:10359000CF92DF92EF92FF920F931F93CF93DF931F
:1035A000C82ED62EB42EC7E0D0E0022F10E087E060
:1035B000E82EF12CBB2059F497012C1B3D0BC801C0
:1035C00002C0959587952A95E2F79C0107C098015E
:1035D0000C2E02C0359527950A94E2F7622F617090
:1035E0008C2D0E948B198D2D61E00E948B198D2DE1
:1035F00060E00E948B1921979FEFCF3FD907D1F64A
:10360000DF91CF911F910F91FF90EF90DF90CF90BE
:10361000BF900895EF92FF920F931F937B018C014F
:1036200020E030E040E05FE40E94861E87FD11C08C
:10363000C801B70120E030E040E05FE40E94AD1C2B
:103640000E94461F9B01AC01205030404040504832
:1036500006C0C801B7010E94461F9B01AC01B90119
:10366000CA011F910F91FF90EF900895A0E0B0E084
:10367000ECE3FBE10C948122FC01EA0180818230C1
:1036800008F438C1DB019C91923008F430C18430D9
:1036900059F4943009F02EC1918111968C911197B3
:1036A000981709F021C126C1943009F420C1923045
:1036B000B1F4823009F01EC1CA01AF0128E0DA017D
:1036C0000D90AD01DC010D92CD012150C1F7DB0160
:1036D00011968C9111979181892389830AC1823037
:1036E00009F405C1C280D380DB0112966D907C90F5
:1036F000139724813581468157811496ED90FD9072
:103700000D911C911797C601861997095C0197FFC7
:1037100004C0AA24BB24A81AB90AB0E2AB16B104AB
:103720000CF061C0181619066CF5370148010A2C17
:1037300004C096948794779467940A94D2F781E0B2
:1037400090E0A0E0B0E00A2C04C0880F991FAA1FE7
:10375000BB1F0A94D2F70197A109B1098E219F21BD
:10376000A023B123EE24FF248701E3940097A10551
:10377000B10519F4EE24FF248701E628F72808296B
:1037800019293CC00097D1F1CA0CDB1C39014A0150
:103790000A2C04C096948794779467940A94D2F77D
:1037A00081E090E0A0E0B0E00A2C04C0880F991FEF
:1037B000AA1FBB1F0A94D2F70197A109B10982235E
:1037C0009323A423B52321E030E040E050E00097AC
:1037D000A105B10519F420E030E0A9012629372917
:1037E000482959290BC06C147D0424F4EE24FF24CD
:1037F000870104C0630120E030E0A9018181FB0161
:103800009181891709F445C0882349F0D801C7017F
:10381000821B930BA40BB50B9C01AD0104C02E19A8
:103820003F09400B510B57FD04C01982DB82CA824D
:103830000BC081E08983DB82CA8250954095309528
:1038400021953F4F4F4F5F4F2C833D834E835F83C6
:103850000DC0880F991FAA1FBB1F8C839D83AE8349
:10386000BF838A819B8101979B838A838C819D8101
:10387000AE81BF819C01AD0121503040404050409D
:103880002F3FEFEF3E07EFEF4E07EFE35E0708F342
:103890000BC08983DB82CA822E0D3F1D401F511F42
:1038A0002C833D834E835F8383E088832C813D811D
:1038B0004E815F8157FF1DC0DA01C9018170907090
:1038C000A070B0705695479537952795822B932B0E
:1038D000A42BB52B8C839D83AE83BF838A819B8170
:1038E00001969B838A8305C0EEEAF1E003C0FB01E9
:1038F00001C0FE01CF01CDB7DEB7EEE00C949D22F2
:10390000A0E2B0E0E6E8FCE10C94892269837A83C6
:103910008B839C832D833E834F83588789E0E82ED9
:10392000F12CEC0EFD1ECE010196B7010E9438214C
:103930008E010F5E1F4FCE010596B8010E943821FF
:10394000C701B801AE01475E5F4F0E94361B0E945F
:103950006A20A096E6E00C94A522A0E2B0E0E3EB9A
:10396000FCE10C94892269837A838B839C832D8369
:103970003E834F8358878E01075F1F4FCE0101960C
:10398000B8010E94382191E1E92EF12CEC0EFD1EC8
:10399000CE010596B7010E9438218A8991E08927D6
:1039A0008A8BC801B701AE01475E5F4F0E94361B8C
:1039B0000E946A20A096E6E00C94A522A0E2B0E066
:1039C000E4EEFCE10C947D2269837A838B839C83F3
:1039D0002D833E834F835887CE010196BE01675FDA
:1039E0007F4F0E943821CE010596BE016F5E7F4F4A
:1039F0000E9438219985923078F089898230C0F010
:103A0000943019F4823041F4CBC0843019F49230F0
:103A100079F4C6C0923051F481E02A859A89291739
:103A200009F480E08A87CE010996BCC0823051F447
:103A300081E02A859A89291709F480E08A8BCE01D2
:103A40004196B0C06D847E848F849888ED88FE880E
:103A50000F89188DE0E2F0E080E090E0DC01AA241C
:103A6000BB24650120E030E0A901B30161707070F2
:103A700061157105D1F02E0D3F1D401F511F15011D
:103A80002601280E391E4A1E5B1E81E090E0A0E050
:103A9000B0E02E153F054007510718F080E090E098
:103AA000DC01820D931DA41DB51DAA0CBB1CCC1CF2
:103AB000DD1C17FF09C061E0262E312C412C512C52
:103AC000A228B328C428D528319749F0EE0CFF1C52
:103AD000001F111F9694879477946794C6CF6B89C3
:103AE0007C89EB85FC856E0F7F1F6E5F7F4F7C8F1F
:103AF0006B8F61E0EA857A89E71709F460E06A8FE5
:103B00006B8D7C8D10C0FC01E170F070309729F056
:103B100056954795379527955068B695A7959795EB
:103B200087956F5F7F4FB7FDEECF0CC0880F991F51
:103B3000AA1FBB1F57FD8160220F331F441F551F53
:103B4000615070408030E0E09E07E0E0AE07E0E4C6
:103B5000BE0760F36B8F7C8F6FE7E62EF12C012D93
:103B6000112DE822F9220A231B2360E4E616F10452
:103B70000105110561F487FD0AC0211531054105D4
:103B8000510529F0805C9F4FAF4FBF4F80788D8FDC
:103B90009E8FAF8FB8A383E0898FCE01499602C074
:103BA0008EEA91E00E946A20A096E2E10C949922AC
:103BB000A8E1B0E0EEEDFDE10C94852269837A8303
:103BC0008B839C832D833E834F8358878E01075FB1
:103BD0001F4FCE010196B8010E94382181E1E82EE5
:103BE000F12CEC0EFD1ECE010596B7010E94382186
:103BF0009985923008F483C08989823008F47BC0AB
:103C00002A853A8923272A87943011F0923021F4AB
:103C1000981709F06CC071C0843039F41D861E8677
:103C20001F86188A1C861B866AC0823019F484E0BD
:103C3000898765C08B859C852B893C89821B930B6A
:103C40009C878B872D853E854F855889ED88FE881A
:103C50000F89188D2E153F054007510738F4220FA4
:103C6000331F441F551F01979C878B876FE170E0BE
:103C7000A12CB12CC12CA0E4DA2E80E090E0DC0174
:103C80002E153F054007510740F08A299B29AC2992
:103C9000BD292E193F09400B510BD694C794B794F8
:103CA000A794220F331F441F551F6150704041F7E6
:103CB0006FE7E62EF12C012D112DE822F9220A23BF
:103CC0001B2360E4E616F1040105110561F487FD8C
:103CD0000AC0211531054105510529F0805C9F4F2F
:103CE000AF4FBF4F80788D879E87AF87B88B8E018F
:103CF000075F1F4F04C0870102C00EEA11E0C80130
:103D00000E946A206896EAE00C94A122A8E1B0E043
:103D1000ECE8FEE10C94892269837A838B839C838F
:103D20002D833E834F8358878E01075F1F4FCE013F
:103D30000196B8010E94382181E1E82EF12CEC0EA9
:103D4000FD1ECE010596B7010E943821898582307B
:103D500040F08989823028F0C801B7010E94A12172
:103D600001C08FEF6896E6E00C94A522A8E1B0E0D0
:103D7000ECEBFEE10C94892269837A838B839C832C
:103D80002D833E834F8358878E01075F1F4FCE01DF
:103D90000196B8010E94382181E1E82EF12CEC0E49
:103DA000FD1ECE010596B7010E943821898582301B
:103DB00040F08989823028F0C801B7010E94A12112
:103DC00001C081E06896E6E00C94A522A8E0B0E08E
:103DD000ECEEFEE10C9489227B018C0183E0898367
:103DE000D801C7018827B7FD83959927AA27BB2744
:103DF000282F8A83E114F1040105110519F482E0EA
:103E0000898337C08EE190E09C838B83222389F0E5
:103E100080E0E81680E0F80680E0080780E81807F0
:103E200069F110950095F094E094E11CF11C011DDE
:103E3000111DED82FE820F831887C801B7010E9411
:103E400010209C01215030401216130694F4022ECB
:103E500004C0EE0CFF1C001F111F0A94D2F7ED8264
:103E6000FE820F8318878EE190E0821B930B9C8368
:103E70008B83CE0101960E946A2004C060E070E04E
:103E800080E09FEC2896E6E00C94A522ACE0B0E040
:103E9000ECE4FFE10C948D2269837A838B839C830D
:103EA000CE010196BE016B5F7F4F0E9438218D814C
:103EB000823081F1823070F1843021F48E81882348
:103EC00069F10AC02F81388537FD24C06E812F31FA
:103ED00031053CF0662311F120E030E040E050E88D
:103EE00021C08EE190E0821B930B29853A854B859A
:103EF0005C8504C056954795379527958A95D2F7E6
:103F0000662381F050954095309521953F4F4F4F56
:103F10005F4F08C020E030E0A90104C02FEF3FEF61
:103F20004FEF5FE7B901CA012C96E2E00C94A92299
:103F3000A8E0B0E0EEE9FFE10C9487227B018C0160
:103F40001A82611571058105910519F482E0898352
:103F50005FC083E089838EE1C82ED12CDC82CB82C6
:103F6000ED82FE820F831887C801B7010E941020DE
:103F7000FC013197F7FF3AC0AA27BB27AE1BBF0B46
:103F800021E030E040E050E00A2E04C0220F331F51
:103F9000441F551F0A94D2F72150304040405040F2
:103FA0002E213F214023512361E070E080E090E02A
:103FB000211531054105510519F460E070E0CB0190
:103FC00004C016950795F794E794AA95D2F7E62AC8
:103FD000F72A082B192BED82FE820F8318878EE1BA
:103FE00090E08E1B9F0B9C838B8312C0309781F0D7
:103FF0000E2E04C0EE0CFF1C001F111F0A94D2F7F6
:10400000ED82FE820F831887CE1ADF0ADC82CB8214
:10401000CE0101960E946A202896E8E00C94A32223
:10402000AF92BF92CF92DF92EF92FF920F931F93C6
:104030007B018C0180E0E81680E0F80681E008074B
:1040400080E0180758F4EFEFEE16F10401051105B2
:1040500009F090F480E090E0DC0117C0F0E0EF168A
:10406000F0E0FF06F0E00F07F1E01F0750F480E1F9
:1040700090E0A0E0B0E009C088E090E0A0E0B0E00F
:1040800004C088E190E0A0E0B0E020E230E040E051
:1040900050E0281B390B4A0B5B0B5701680104C029
:1040A000D694C794B794A7948A95D2F7D601C50140
:1040B0008A549E4FFC018081281B31094109510916
:1040C000C9011F910F91FF90EF90DF90CF90BF90AB
:1040D000AF900895EF92FF920F931F93CF93DF93CA
:1040E000FC01248135814681578161818081823044
:1040F00020F44061EFEFF0E0A3C0843009F49BC0EE
:10410000823009F492C0211531054105510509F4A9
:104110008FC00280F381E02D8FEFE238F8070CF0BA
:104120005AC0C2E8DFEFCE1BDF0BCA31D1056CF5F8
:1041300079018A010C2E04C016950795F794E7942F
:104140000A94D2F781E090E0A0E0B0E00C2E04C029
:10415000880F991FAA1FBB1F0A94D2F70197A109C4
:10416000B10982239323A423B52321E030E040E06A
:1041700050E00097A105B10519F420E030E0A90155
:104180002E293F29402B512B03C020E030E0A9010C
:10419000DA01C9018F779070A070B07080349105FA
:1041A000A105B10539F427FF09C0205C3F4F4F4FEF
:1041B0005F4F04C0215C3F4F4F4F5F4FE1E0F0E0A5
:1041C000203080E0380780E0480780E4580728F571
:1041D000E0E0F0E022C0E038F1056CF5E158FF4F77
:1041E000DA01C9018F779070A070B07080349105AA
:1041F000A105B10539F427FF09C0205C3F4F4F4F9F
:104200005F4F04C0215C3F4F4F4F5F4F57FF05C0CA
:104210005695479537952795319687E0569547955A
:10422000379527958A95D1F70BC0E0E0F0E005C0FF
:10423000E0E0F0E005C0EFEFF0E020E030E0A901C1
:104240008E2F879588278795942F9F776795662768
:104250006795E695E22EA92FA82BFE2FF62B622F4D
:10426000732F8A2F9F2FCDB7DEB7E6E00C94A522DF
:10427000DC01FB012C9111963C91119712968C91C7
:104280001297482F4F7750E0982F991F9927991F21
:1042900013966C911397862F880F892B90E0661FD9
:1042A0006627661F6183009739F5211531054105A1
:1042B000510511F482E029C082E89FEF9383828345
:1042C00067E0220F331F441F551F6A95D1F783E023
:1042D000808309C0220F331F441F551F82819381A1
:1042E000019793838283203080E0380780E048077D
:1042F00080E4580778F320C08F3F910579F42115A9
:1043000031054105510519F484E08083089544FF87
:1043100003C081E0808310C010820EC08F57904090
:104320009383828383E0808387E0220F331F441FBF
:10433000551F8A95D1F7506424833583468357836C
:104340000895FC01DB019081923008F449C08C9102
:10435000823008F445C0943051F461818430B1F565
:1043600011962C91119730E0261B310941C0843001
:1043700021F0923041F48230B1F111968C91119775
:104380008823A1F12DC06181823001F111968C91B9
:1043900011976817D9F42281338112968D919C91DF
:1043A00013978217930794F028173907BCF02481DC
:1043B00035814681578114968D919D910D90BC91C8
:1043C000A02D82179307A407B50718F4662341F0C0
:1043D0000DC0281739074A075B0728F4662331F018
:1043E00021E030E005C020E030E002C02FEF3FEFD9
:1043F000C9010895629FD001739FF001829FE00D73
:10440000F11D649FE00DF11D929FF00D839FF00D53
:10441000749FF00D659FF00D9927729FB00DE11DFF
:10442000F91F639FB00DE11DF91FBD01CF011124DC
:10443000089597FB092E07260AD077FD04D049D0AE
:1044400006D000201AF4709561957F4F0895F6F715
:10445000909581959F4F0895A1E21A2EAA1BBB1B30
:10446000FD010DC0AA1FBB1FEE1FFF1FA217B30740
:10447000E407F50720F0A21BB30BE40BF50B661F56
:10448000771F881F991F1A9469F76095709580951A
:1044900090959B01AC01BD01CF01089597FB092EBA
:1044A00005260ED057FD04D0D7DF0AD0001C38F403
:1044B00050954095309521953F4F4F4F5F4F089550
:1044C000F6F790958095709561957F4F8F4F9F4F30
:1044D0000895AA1BBB1B51E107C0AA1FBB1FA6174B
:1044E000B70710F0A61BB70B881F991F5A95A9F79D
:1044F00080959095BC01CD0108952F923F924F92E7
:104500005F926F927F928F929F92AF92BF92CF9263
:10451000DF92EF92FF920F931F93CF93DF93CDB76C
:10452000DEB7CA1BDB0B0FB6F894DEBF0FBECDBFE4
:1045300009942A88398848885F846E847D848C84B5
:104540009B84AA84B984C884DF80EE80FD800C81BE
:104550001B81AA81B981CE0FD11D0FB6F894DEBFA1
:104560000FBECDBFED010895EE0FFF1F0590F49132
:10457000E02D0994CF93DF938230910510F482E00F
:1045800090E0E091AC03F091AD0340E050E020E01A
:1045900030E026C06081718168177907E0F0681704
:1045A000790781F4828193812115310531F0D90198
:1045B00013969C938E9312972BC09093AD03809388
:1045C000AC0326C04115510519F06417750718F49E
:1045D000AB01E901DF019F0172816381E72FF62FB3
:1045E0003097C1F64115510501F1481B590B443074
:1045F000510580F412968D919C911397209719F094
:104600009B838A8304C09093AD038093AC03FD0128
:10461000329646C0FD01E40FF51F819391934250FD
:10462000504011965C934E933BC02091AA03309169
:10463000AB032115310541F42091B8023091B90244
:104640003093AB032093AA032091BA023091BB02AE
:104650002115310541F42DB73EB74091B602509176
:10466000B702241B350BE091AA03F091AB03E217CC
:10467000F307A0F42E1B3F0B2817390778F0AC0185
:104680004E5F5F4F2417350748F04E0F5F1F509362
:10469000AB034093AA038193919302C0E0E0F0E062
:1046A000CF01DF91CF910895CF93DF93009709F465
:1046B00091C0FC013297138212826091AC03709119
:1046C000AD036115710581F420813181280F391FF7
:1046D0008091AA039091AB038217930799F5F09309
:1046E000AB03E093AA0376C0DB0180E090E002C058
:1046F000CD01D901AE17BF0748F412962D913C9118
:10470000139721153105A1F7CD0121C0B383A283F1
:10471000EF01499159919E01240F351FA217B3074C
:1047200079F42D913C911197240F351F2E5F3F4F47
:104730003183208312962D913C91139733832283EA
:10474000009729F4F093AD03E093AC0343C0DC0180
:104750001396FC93EE9312974D915D91A40FB51FA4
:10476000EA17FB0769F420813181240F351F2E5F82
:104770003F4FEC0139832883228133813B832A8395
:10478000E0E0F0E002C0FB01BC01DB0112968D917C
:104790009C9113970097B9F79B012E5F3F4F8D9126
:1047A0009C911197820F931F4091AA035091AB03E4
:1047B0004817590779F4309729F41092AD031092F5
:1047C000AC0302C013821282225030403093AB03FC
:1047D0002093AA03DF91CF910895A0E0B0E0E3EF2A
:1047E000F3E20C948522EC01688179818A819B81B6
:1047F000611571058105910521F464E279ED8BE580
:1048000097E02DE133EF41E050E00E944E22790124
:104810008A0127EA31E440E050E00E94FA215B017E
:104820006C01C801B7012CEE34EF4FEF5FEF0E942F
:10483000FA219B01AC012A0D3B1D4C1D5D1D57FF4C
:1048400004C02150304040405048288339834A8377
:104850005B835F77B901CA01CDB7DEB7EAE00C949C
:10486000A1220E94ED2308958CEB92E00E94ED239B
:1048700008956093BC027093BD028093BE02909332
:10488000BF020895A0E0B0E0E8E4F4E20C948322D3
:104890008C01CB010115110529F40E94BA22082FC1
:1048A000192FB5C0D80112979801260F371F2A1764
:1048B0003B0708F4AAC0ED90FC901197E616F706A6
:1048C000D0F045E0E416F10408F4A1C0A70144507B
:1048D00050404617570708F49AC0A701425050406D
:1048E000461B570BF901419351936D937C93CF0174
:1048F0000E9454238CC05B01AE18BF0848018E0C87
:104900009F1CE091AC03F091AD03CC24DD24C0E00A
:10491000D0E041C0E815F90599F560817181AB01DE
:104920004E5F5F4F4A155B0558F1AB014A195B09B1
:10493000CC24DD246894C1F8C40ED51E8280A380E7
:10494000E5E0CE16D10448F0F9018282A3825183BA
:10495000408311969C938E9309C0C7010296860FDF
:10496000971F11969C938E93E82DFA2D209719F09E
:10497000FB83EA834CC0F093AD03E093AC0347C0E4
:1049800040815181C416D50608F46A01EF015281B5
:104990004381E52FF42F309709F0BCCF4091AA0353
:1049A0005091AB0348155905E9F4C816D906D0F45F
:1049B0004091BA025091BB024115510541F44DB7E7
:1049C0005EB76091B6027091B702461B570B241771
:1049D0003507D8F43093AB032093AA0311969C9328
:1049E0008E9315C00E94BA22C82EE6016E01D92E00
:1049F000E601209751F08C2DB801A7010E9459259E
:104A0000C8010E945423860102C000E010E0C801E2
:104A1000CDB7DEB7ECE00C949F221F93FC019927E1
:104A20008827BC01E89411911032E9F3193010F095
:104A30001E30C8F31B3251F01D3249F4689406C091
:104A40000E942626610F711D811D911D1191105329
:104A50001A30B0F33EF490958095709561957F4F34
:104A60008F4F9F4F1F910895911140C1803219F0CF
:104A700089508550D0F708959111089581548A5135
:104A800008F4805E855A08959111089581568A51DF
:104A900008F4805285580895FB01DC0104C08D9113
:104AA0000190801921F441505040C8F7881B990BA0
:104AB0000895FB01DC0102C001900D92415050406D
:104AC000D8F708956817790768F4FB01DC01E40F53
:104AD000F51FA40FB51F02C002900E924150504026
:104AE000D8F708950C945925FC018191861721F07F
:104AF0008823D9F7992708953197CF010895FB01AD
:104B0000DC018D91019080190110D9F3990B089562
:104B1000FB01DC0101900D920020E1F70895FB01FB
:104B2000DC014150504030F08D910190801919F412
:104B30000020B9F7881B990B0895FB01DC01415057
:104B4000504048F001900D920020C9F701C01D921D
:104B500041505040E0F70895FC0181E090E0019061
:104B6000061609F4CF010020D1F701970895FB0143
:104B700051915523A9F0BF01DC014D914517411119
:104B8000E1F759F4CD010190002049F04D91401515
:104B90004111C9F3FB014111EFCF81E090E0019792
:104BA0000895FB019F01E8944230C4F04532B4F40B
:104BB0004A3029F497FB1EF4909581959F4F642FFE
:104BC00077270E946922805D8A330CF0895D81938A
:104BD000CB010097A1F716F45DE251931082C90151
:104BE0000C947926FA01CF93FF93EF93223044F18E
:104BF000253234F5C22FE894CA3049F497FB3EF4CD
:104C000090958095709561957F4F8F4F9F4F2C2F7A
:104C1000332744275527FF93EF930E942C22EF91CF
:104C2000FF91605D6A330CF0695D6193B901CA015F
:104C3000605070408040904051F716F4CDE2C1932F
:104C400010828F919F91CF910C947926592F482FE4
:104C5000372F262F660F771F881F991F660F771F24
:104C6000881F991F620F731F841F951F660F771F80
:104C7000881F991F0895FA01CF93FF93EF93223075
:104C8000CCF02532BCF4C22F2C2F332744275527D4
:104C9000FF93EF930E942C22EF91FF91605D6A33A6
:104CA0000CF0695D6193B901CA01605070408040A9
:104CB000904051F710828F919F91CF910C9479265B
:104CC000FB019F01423074F0453264F4642F772772
:104CD0000E946922805D8A330CF0895D8193CB014B
:104CE0000097A1F71082C9010C947926992788278B
:104CF0000895DC01FC01672F71917723E1F732976A
:104D000004C07C916D9370836291AE17BF07C8F3A6
:064D10000895F894FFCFA6
:104D16000D0A2B494E513D310D0A000D0A2B5354F5
:104D2600574D4F443D300D0A000D0A2B53544E414A
:104D36003D4164617074696373456C65637469634E
:104D46000D0A000D0A2B53544F4155543D310D0A9F
:104D5600000D0A2B53544155544F3D300D0A000D9A
:104D66000A202B535450494E3D303030300D0A0046
:104D76000D0A2B4C4F53535245434F4E4E3D300D6B
:104D86000A0007F0000000000078034E06130342F5
:104D9600032603640300000000C1174E06C117C1B5
:104DA60017C117C11700000000A60500000000C1CA
:104DB600172E0000000000C1174E06FF000100007C
:104DC60000000000000000010202030303030404C4
:104DD6000404040404040505050505050505050583
:104DE6000505050505050606060606060606060663
:104DF600060606060606060606060606060606064D
:104E06000606060606060707070707070707070732
:104E1600070707070707070707070707070707071C
:104E2600070707070707070707070707070707070C
:104E360007070707070707070707070707070707FC
:104E460007070707070708080808080808080808E2
:104E560008080808080808080808080808080808CC
:104E660008080808080808080808080808080808BC
:104E760008080808080808080808080808080808AC
:104E8600080808080808080808080808080808089C
:104E9600080808080808080808080808080808088C
:104EA600080808080808080808080808080808087C
:104EB600080808080808080808080808080808086C
:104EC6000808080808082000AE03000001000000DA
:00000001FF
